 StackTrace

 Timestamp is 105e7723 (reproducible build file hash)

 Preferred load address is 0000000180000000

 Start         Length     Name                   Class
 0001:00000000 00003190H .text$mn                CODE
 0001:00003190 00000036H .text$mn$00             CODE
 0001:000031c6 00000092H .text$x                 CODE
 0002:00000000 00000198H .idata$5                DATA
 0002:00000198 00000038H .00cfg                  DATA
 0002:000001d0 00000008H .CRT$XCA                DATA
 0002:000001d8 00000008H .CRT$XCZ                DATA
 0002:000001e0 00000008H .CRT$XIA                DATA
 0002:000001e8 00000008H .CRT$XIC                DATA
 0002:000001f0 00000008H .CRT$XIZ                DATA
 0002:000001f8 00000008H .CRT$XLA                DATA
 0002:00000200 00000008H .CRT$XLZ                DATA
 0002:00000208 00000008H .CRT$XPA                DATA
 0002:00000210 00000008H .CRT$XPZ                DATA
 0002:00000218 00000008H .CRT$XTA                DATA
 0002:00000220 00000010H .CRT$XTZ                DATA
 0002:00000228 00000000H .gehcont$y              DATA
 0002:00000228 00000000H .gfids$y                DATA
 0002:00000230 00001dd0H .rdata                  DATA
 0002:00002000 00000000H .rdata$CastGuardVftablesA DATA
 0002:00002000 00000000H .rdata$CastGuardVftablesC DATA
 0002:00002000 00000028H .rdata$T                DATA
 0002:00002028 000000a4H .rdata$voltmd           DATA
 0002:000020cc 0000031cH .rdata$zzzdbg           DATA
 0002:000023e8 00000008H .rtc$IAA                DATA
 0002:000023f0 00000008H .rtc$IZZ                DATA
 0002:000023f8 00000008H .rtc$TAA                DATA
 0002:00002400 00000008H .rtc$TZZ                DATA
 0002:00002408 00000004H .tls                    DATA
 0002:0000240c 00000004H .tls$                   DATA
 0002:00002410 00000008H .tls$ZZZ                DATA
 0002:00002418 00000318H .xdata                  DATA
 0002:00002730 000005b4H .edata                  DATA
 0002:00002ce4 00000064H .idata$2                DATA
 0002:00002d48 00000018H .idata$3                DATA
 0002:00002d60 00000198H .idata$4                DATA
 0002:00002ef8 0000041eH .idata$6                DATA
 0003:00000000 00000080H .data                   DATA
 0003:00000080 0001f168H .bss                    DATA
 0004:00000000 000003d8H .pdata                  DATA

  Address         Publics by Value              Rva+Base               Lib:Object

 0000:00000000       __AbsoluteZero             0000000000000000     <absolute>
 0000:00000000       ___safe_se_handler_count   0000000000000000     <absolute>
 0000:00000000       ___safe_se_handler_table   0000000000000000     <absolute>
 0000:00000000       __arm64x_extra_rfe_table   0000000000000000     <absolute>
 0000:00000000       __arm64x_extra_rfe_table_size 0000000000000000     <absolute>
 0000:00000000       __arm64x_native_entrypoint 0000000000000000     <absolute>
 0000:00000000       __arm64x_redirection_metadata 0000000000000000     <absolute>
 0000:00000000       __arm64x_redirection_metadata_count 0000000000000000     <absolute>
 0000:00000000       __dynamic_value_reloc_table 0000000000000000     <absolute>
 0000:00000000       __enclave_config           0000000000000000     <absolute>
 0000:00000000       __guard_check_icall_a64n_fptr 0000000000000000     <absolute>
 0000:00000000       __guard_eh_cont_count      0000000000000000     <absolute>
 0000:00000000       __guard_eh_cont_table      0000000000000000     <absolute>
 0000:00000000       __guard_fids_count         0000000000000000     <absolute>
 0000:00000000       __guard_fids_table         0000000000000000     <absolute>
 0000:00000000       __guard_iat_count          0000000000000000     <absolute>
 0000:00000000       __guard_iat_table          0000000000000000     <absolute>
 0000:00000000       __guard_longjmp_count      0000000000000000     <absolute>
 0000:00000000       __guard_longjmp_table      0000000000000000     <absolute>
 0000:00000000       __hybrid_auxiliary_iat     0000000000000000     <absolute>
 0000:00000000       __hybrid_auxiliary_iat_copy 0000000000000000     <absolute>
 0000:00000000       __hybrid_code_map          0000000000000000     <absolute>
 0000:00000000       __hybrid_code_map_count    0000000000000000     <absolute>
 0000:00000000       __x64_code_ranges_to_entry_points 0000000000000000     <absolute>
 0000:00000000       __x64_code_ranges_to_entry_points_count 0000000000000000     <absolute>
 0000:00000100       __guard_flags              0000000000000100     <absolute>
 0000:00000000       __ImageBase                0000000180000000     <linker-defined>
 0001:00000000       ?NewObject@JNIEnv_@@QEAAPEAV_jobject@@PEAV_jclass@@PEAU_jmethodID@@ZZ 0000000180001000 f i libStackTrace.obj
 0001:00000028       ?TranslateError@@YAPEBDW4jvmtiError@@@Z 0000000180001028 f   libStackTrace.obj
 0001:000002e0       ?nsk_jni_check_exception@@YAHPEAUJNIEnv_@@QEBDH@Z 00000001800012e0 f   libStackTrace.obj
 0001:00000424       ?nsk_jni_lverify@@YAHHPEAUJNIEnv_@@HQEBDH1ZZ 0000000180001424 f   libStackTrace.obj
 0001:000004c4       Agent_Initialize           00000001800014c4 f   libStackTrace.obj
 0001:000005a8       Agent_OnAttach             00000001800015a8 f   libStackTrace.obj
 0001:000005a8       Agent_OnLoad               00000001800015a8 f   libStackTrace.obj
 0001:000005b0       Java_nsk_jvmti_unit_FollowReferences_FollowRefObjects_addRefToVerify 00000001800015b0 f   libStackTrace.obj
 0001:00000788       Java_nsk_jvmti_unit_FollowReferences_FollowRefObjects_getTag 0000000180001788 f   libStackTrace.obj
 0001:00000848       Java_nsk_jvmti_unit_FollowReferences_FollowRefObjects_resetRefsToVerify 0000000180001848 f   libStackTrace.obj
 0001:00000850       Java_nsk_jvmti_unit_FollowReferences_FollowRefObjects_resetTags 0000000180001850 f   libStackTrace.obj
 0001:00000894       Java_nsk_jvmti_unit_FollowReferences_FollowRefObjects_setTag 0000000180001894 f   libStackTrace.obj
 0001:00000aec       Java_nsk_jvmti_unit_StackTrace_JvmtiTest_CreateRawMonitor 0000000180001aec f   libStackTrace.obj
 0001:00000b88       Java_nsk_jvmti_unit_StackTrace_JvmtiTest_GetFrameCount 0000000180001b88 f   libStackTrace.obj
 0001:00000bdc       Java_nsk_jvmti_unit_StackTrace_JvmtiTest_GetResult 0000000180001bdc f   libStackTrace.obj
 0001:00000be4       Java_nsk_jvmti_unit_StackTrace_JvmtiTest_GetStackTrace 0000000180001be4 f   libStackTrace.obj
 0001:00001044       Java_nsk_jvmti_unit_StackTrace_JvmtiTest_RawMonitorEnter 0000000180002044 f   libStackTrace.obj
 0001:0000109c       Java_nsk_jvmti_unit_StackTrace_JvmtiTest_RawMonitorExit 000000018000209c f   libStackTrace.obj
 0001:000010f4       Java_nsk_jvmti_unit_StackTrace_JvmtiTest_RawMonitorNotify 00000001800020f4 f   libStackTrace.obj
 0001:0000114c       Java_nsk_jvmti_unit_StackTrace_JvmtiTest_RawMonitorWait 000000018000214c f   libStackTrace.obj
 0001:000011a8       Java_nsk_jvmti_unit_StackTrace_JvmtiTest_SaveThreadInfo 00000001800021a8 f   libStackTrace.obj
 0001:000011a8       _guard_check_icall_nop     00000001800021a8 f   MSVCRT:guard_support.obj
 0001:000011ac       Java_nsk_share_jvmti_ArgumentHandler_getAgentOptionsString 00000001800021ac f   libStackTrace.obj
 0001:0000125c       Java_nsk_share_jvmti_DebugeeClass_checkStatus 000000018000225c f   libStackTrace.obj
 0001:000012e4       Java_nsk_share_jvmti_DebugeeClass_resetAgentData 00000001800022e4 f   libStackTrace.obj
 0001:00001344       Java_nsk_share_jvmti_RedefineAgent_agentStatus 0000000180002344 f   libStackTrace.obj
 0001:00001350       Java_nsk_share_jvmti_RedefineAgent_isRedefined 0000000180002350 f   libStackTrace.obj
 0001:0000135c       Java_nsk_share_jvmti_RedefineAgent_redefineAttempted 000000018000235c f   libStackTrace.obj
 0001:00001368       MA_checkStatus             0000000180002368 f   libStackTrace.obj
 0001:0000140c       __local_stdio_printf_options 000000018000240c f i libStackTrace.obj
 0001:00001414       _snprintf                  0000000180002414 f i libStackTrace.obj
 0001:00001644       debug_printf               0000000180002644 f   libStackTrace.obj
 0001:000016a0       exitOnError                00000001800026a0 f   libStackTrace.obj
 0001:00001754       fprintf                    0000000180002754 f i libStackTrace.obj
 0001:00001798       nsk_jvmti_lverify          0000000180002798 f   libStackTrace.obj
 0001:00001888       nsk_jvmti_resetAgentData   0000000180002888 f   libStackTrace.obj
 0001:00001908       nsk_jvmti_setFailStatus    0000000180002908 f   libStackTrace.obj
 0001:00001944       nsk_lcomplain              0000000180002944 f   libStackTrace.obj
 0001:00001964       nsk_ldisplay               0000000180002964 f   libStackTrace.obj
 0001:00001984       nsk_ltrace                 0000000180002984 f   libStackTrace.obj
 0001:000019a4       nsk_lvcomplain             00000001800029a4 f   libStackTrace.obj
 0001:00001b5c       nsk_lvdisplay              0000000180002b5c f   libStackTrace.obj
 0001:00001ba8       nsk_lverify                0000000180002ba8 f   libStackTrace.obj
 0001:00001c04       nsk_lvtrace                0000000180002c04 f   libStackTrace.obj
 0001:00001c64       nsk_printf                 0000000180002c64 f   libStackTrace.obj
 0001:00001c8c       nsk_vprintf                0000000180002c8c f   libStackTrace.obj
 0001:00001d40       printf                     0000000180002d40 f i libStackTrace.obj
 0001:00002268       __raise_securityfailure    0000000180003268 f   MSVCRT:gs_report.obj
 0001:0000229c       __report_gsfailure         000000018000329c f   MSVCRT:gs_report.obj
 0001:000024dc       __GSHandlerCheck           00000001800034dc f   MSVCRT:gshandler.obj
 0001:000024fc       __GSHandlerCheckCommon     00000001800034fc f   MSVCRT:gshandler.obj
 0001:00002570       __security_check_cookie    0000000180003570 f   MSVCRT:amdsecgs.obj
 0001:000028b0       _DllMainCRTStartup         00000001800038b0 f   MSVCRT:dll_dllmain.obj
 0001:000028f0       __scrt_acquire_startup_lock 00000001800038f0 f   MSVCRT:utility.obj
 0001:0000292c       __scrt_dllmain_after_initialize_c 000000018000392c f   MSVCRT:utility.obj
 0001:00002960       __scrt_dllmain_before_initialize_c 0000000180003960 f   MSVCRT:utility.obj
 0001:00002978       __scrt_dllmain_crt_thread_attach 0000000180003978 f   MSVCRT:utility.obj
 0001:000029a0       __scrt_dllmain_crt_thread_detach 00000001800039a0 f   MSVCRT:utility.obj
 0001:000029b8       __scrt_dllmain_exception_filter 00000001800039b8 f   MSVCRT:utility.obj
 0001:00002a18       __scrt_dllmain_uninitialize_c 0000000180003a18 f   MSVCRT:utility.obj
 0001:00002a48       __scrt_dllmain_uninitialize_critical 0000000180003a48 f   MSVCRT:utility.obj
 0001:00002a5c       __scrt_initialize_crt      0000000180003a5c f   MSVCRT:utility.obj
 0001:00002aa8       __scrt_initialize_onexit_tables 0000000180003aa8 f   MSVCRT:utility.obj
 0001:00002b34       __scrt_is_nonwritable_in_current_image 0000000180003b34 f   MSVCRT:utility.obj
 0001:00002bcc       __scrt_release_startup_lock 0000000180003bcc f   MSVCRT:utility.obj
 0001:00002bf0       __scrt_uninitialize_crt    0000000180003bf0 f   MSVCRT:utility.obj
 0001:00002c1c       _onexit                    0000000180003c1c f   MSVCRT:utility.obj
 0001:00002c58       atexit                     0000000180003c58 f   MSVCRT:utility.obj
 0001:00002c70       __crt_debugger_hook        0000000180003c70 f   MSVCRT:utility_desktop.obj
 0001:00002c78       __scrt_fastfail            0000000180003c78 f   MSVCRT:utility_desktop.obj
 0001:00002dc4       __security_init_cookie     0000000180003dc4 f   MSVCRT:gs_support.obj
 0001:00002e70       DllMain                    0000000180003e70 f   MSVCRT:dll_dllmain_stub.obj
 0001:00002e94       ?__scrt_initialize_type_info@@YAXXZ 0000000180003e94 f   MSVCRT:tncleanup.obj
 0001:00002ea4       ?__scrt_uninitialize_type_info@@YAXXZ 0000000180003ea4 f   MSVCRT:tncleanup.obj
 0001:00002eb0       __local_stdio_scanf_options 0000000180003eb0 f i MSVCRT:default_local_stdio_options.obj
 0001:00002eb8       __scrt_initialize_default_local_stdio_options 0000000180003eb8 f   MSVCRT:default_local_stdio_options.obj
 0001:00002ed4       __scrt_get_dyn_tls_init_callback 0000000180003ed4 f   MSVCRT:dyn_tls_init.obj
 0001:00002edc       _RTC_Initialize            0000000180003edc f   MSVCRT:initsect.obj
 0001:00002f18       _RTC_Terminate             0000000180003f18 f   MSVCRT:initsect.obj
 0001:00002f54       __isa_available_init       0000000180003f54 f   MSVCRT:cpu_disp.obj
 0001:00003100       _get_startup_argv_mode     0000000180004100 f   MSVCRT:argv_mode.obj
 0001:00003108       __scrt_is_ucrt_dll_in_use  0000000180004108 f   MSVCRT:ucrt_detection.obj
 0001:00003120       memcpy                     0000000180004120 f   vcruntime:VCRUNTIME140.dll
 0001:00003126       memset                     0000000180004126 f   vcruntime:VCRUNTIME140.dll
 0001:0000312c       strchr                     000000018000412c f   vcruntime:VCRUNTIME140.dll
 0001:00003132       strstr                     0000000180004132 f   vcruntime:VCRUNTIME140.dll
 0001:00003138       __C_specific_handler       0000000180004138 f   vcruntime:VCRUNTIME140.dll
 0001:0000313e       __std_type_info_destroy_list 000000018000413e f   vcruntime:VCRUNTIME140.dll
 0001:00003144       strlen                     0000000180004144 f   ucrt:api-ms-win-crt-string-l1-1-0.dll
 0001:0000314a       _initterm                  000000018000414a f   ucrt:api-ms-win-crt-runtime-l1-1-0.dll
 0001:00003150       _initterm_e                0000000180004150 f   ucrt:api-ms-win-crt-runtime-l1-1-0.dll
 0001:00003156       _seh_filter_dll            0000000180004156 f   ucrt:api-ms-win-crt-runtime-l1-1-0.dll
 0001:0000315c       _configure_narrow_argv     000000018000415c f   ucrt:api-ms-win-crt-runtime-l1-1-0.dll
 0001:00003162       _initialize_narrow_environment 0000000180004162 f   ucrt:api-ms-win-crt-runtime-l1-1-0.dll
 0001:00003168       _initialize_onexit_table   0000000180004168 f   ucrt:api-ms-win-crt-runtime-l1-1-0.dll
 0001:0000316e       _register_onexit_function  000000018000416e f   ucrt:api-ms-win-crt-runtime-l1-1-0.dll
 0001:00003174       _execute_onexit_table      0000000180004174 f   ucrt:api-ms-win-crt-runtime-l1-1-0.dll
 0001:0000317a       _crt_atexit                000000018000417a f   ucrt:api-ms-win-crt-runtime-l1-1-0.dll
 0001:00003180       _cexit                     0000000180004180 f   ucrt:api-ms-win-crt-runtime-l1-1-0.dll
 0001:00003188       __acrt_initialize          0000000180004188 f   MSVCRT:ucrt_stubs.obj
 0001:00003188       __acrt_thread_attach       0000000180004188 f   MSVCRT:ucrt_stubs.obj
 0001:00003188       __acrt_thread_detach       0000000180004188 f   MSVCRT:ucrt_stubs.obj
 0001:00003188       __acrt_uninitialize        0000000180004188 f   MSVCRT:ucrt_stubs.obj
 0001:00003188       __acrt_uninitialize_critical 0000000180004188 f   MSVCRT:ucrt_stubs.obj
 0001:00003188       __scrt_stub_for_acrt_initialize 0000000180004188 f   MSVCRT:ucrt_stubs.obj
 0001:00003188       __scrt_stub_for_acrt_thread_attach 0000000180004188 f   MSVCRT:ucrt_stubs.obj
 0001:00003188       __scrt_stub_for_acrt_thread_detach 0000000180004188 f   MSVCRT:ucrt_stubs.obj
 0001:00003188       __scrt_stub_for_acrt_uninitialize 0000000180004188 f   MSVCRT:ucrt_stubs.obj
 0001:00003188       __scrt_stub_for_acrt_uninitialize_critical 0000000180004188 f   MSVCRT:ucrt_stubs.obj
 0001:00003188       __vcrt_initialize          0000000180004188 f   MSVCRT:ucrt_stubs.obj
 0001:00003188       __vcrt_thread_attach       0000000180004188 f   MSVCRT:ucrt_stubs.obj
 0001:00003188       __vcrt_thread_detach       0000000180004188 f   MSVCRT:ucrt_stubs.obj
 0001:00003188       __vcrt_uninitialize        0000000180004188 f   MSVCRT:ucrt_stubs.obj
 0001:00003188       __vcrt_uninitialize_critical 0000000180004188 f   MSVCRT:ucrt_stubs.obj
 0001:0000318c       __scrt_stub_for_is_c_termination_complete 000000018000418c f   MSVCRT:ucrt_stubs.obj
 0001:0000318c       _is_c_termination_complete 000000018000418c f   MSVCRT:ucrt_stubs.obj
 0001:000031a0       _guard_dispatch_icall_nop  00000001800041a0 f   MSVCRT:guard_dispatch.obj
 0001:000031c0       _guard_xfg_dispatch_icall_nop 00000001800041c0 f   MSVCRT:guard_xfg_dispatch.obj
 0002:00000000       __imp_RtlCaptureContext    0000000180005000     kernel32:KERNEL32.dll
 0002:00000008       __imp_RtlLookupFunctionEntry 0000000180005008     kernel32:KERNEL32.dll
 0002:00000010       __imp_RtlVirtualUnwind     0000000180005010     kernel32:KERNEL32.dll
 0002:00000018       __imp_UnhandledExceptionFilter 0000000180005018     kernel32:KERNEL32.dll
 0002:00000020       __imp_SetUnhandledExceptionFilter 0000000180005020     kernel32:KERNEL32.dll
 0002:00000028       __imp_GetCurrentProcess    0000000180005028     kernel32:KERNEL32.dll
 0002:00000030       __imp_TerminateProcess     0000000180005030     kernel32:KERNEL32.dll
 0002:00000038       __imp_IsProcessorFeaturePresent 0000000180005038     kernel32:KERNEL32.dll
 0002:00000040       __imp_CloseHandle          0000000180005040     kernel32:KERNEL32.dll
 0002:00000048       __imp_InitializeCriticalSectionAndSpinCount 0000000180005048     kernel32:KERNEL32.dll
 0002:00000050       __imp_DeleteCriticalSection 0000000180005050     kernel32:KERNEL32.dll
 0002:00000058       __imp_CreateEventW         0000000180005058     kernel32:KERNEL32.dll
 0002:00000060       __imp_GetModuleHandleW     0000000180005060     kernel32:KERNEL32.dll
 0002:00000068       __imp_GetProcAddress       0000000180005068     kernel32:KERNEL32.dll
 0002:00000070       __imp_IsDebuggerPresent    0000000180005070     kernel32:KERNEL32.dll
 0002:00000078       __imp_QueryPerformanceCounter 0000000180005078     kernel32:KERNEL32.dll
 0002:00000080       __imp_GetCurrentProcessId  0000000180005080     kernel32:KERNEL32.dll
 0002:00000088       __imp_GetCurrentThreadId   0000000180005088     kernel32:KERNEL32.dll
 0002:00000090       __imp_GetSystemTimeAsFileTime 0000000180005090     kernel32:KERNEL32.dll
 0002:00000098       __imp_DisableThreadLibraryCalls 0000000180005098     kernel32:KERNEL32.dll
 0002:000000a0       __imp_InitializeSListHead  00000001800050a0     kernel32:KERNEL32.dll
 0002:000000a8       \177KERNEL32_NULL_THUNK_DATA 00000001800050a8     kernel32:KERNEL32.dll
 0002:000000b0       __imp_memcpy               00000001800050b0     vcruntime:VCRUNTIME140.dll
 0002:000000b8       __imp_memset               00000001800050b8     vcruntime:VCRUNTIME140.dll
 0002:000000c0       __imp_strchr               00000001800050c0     vcruntime:VCRUNTIME140.dll
 0002:000000c8       __imp_strstr               00000001800050c8     vcruntime:VCRUNTIME140.dll
 0002:000000d0       __imp___C_specific_handler 00000001800050d0     vcruntime:VCRUNTIME140.dll
 0002:000000d8       __imp___std_type_info_destroy_list 00000001800050d8     vcruntime:VCRUNTIME140.dll
 0002:000000e0       \177VCRUNTIME140_NULL_THUNK_DATA 00000001800050e0     vcruntime:VCRUNTIME140.dll
 0002:000000e8       __imp__errno               00000001800050e8     ucrt:api-ms-win-crt-runtime-l1-1-0.dll
 0002:000000f0       __imp_exit                 00000001800050f0     ucrt:api-ms-win-crt-runtime-l1-1-0.dll
 0002:000000f8       __imp__cexit               00000001800050f8     ucrt:api-ms-win-crt-runtime-l1-1-0.dll
 0002:00000100       __imp__crt_atexit          0000000180005100     ucrt:api-ms-win-crt-runtime-l1-1-0.dll
 0002:00000108       __imp__execute_onexit_table 0000000180005108     ucrt:api-ms-win-crt-runtime-l1-1-0.dll
 0002:00000110       __imp__register_onexit_function 0000000180005110     ucrt:api-ms-win-crt-runtime-l1-1-0.dll
 0002:00000118       __imp__initialize_onexit_table 0000000180005118     ucrt:api-ms-win-crt-runtime-l1-1-0.dll
 0002:00000120       __imp__initialize_narrow_environment 0000000180005120     ucrt:api-ms-win-crt-runtime-l1-1-0.dll
 0002:00000128       __imp__configure_narrow_argv 0000000180005128     ucrt:api-ms-win-crt-runtime-l1-1-0.dll
 0002:00000130       __imp__seh_filter_dll      0000000180005130     ucrt:api-ms-win-crt-runtime-l1-1-0.dll
 0002:00000138       __imp__initterm_e          0000000180005138     ucrt:api-ms-win-crt-runtime-l1-1-0.dll
 0002:00000140       __imp__initterm            0000000180005140     ucrt:api-ms-win-crt-runtime-l1-1-0.dll
 0002:00000148       \177api-ms-win-crt-runtime-l1-1-0_NULL_THUNK_DATA 0000000180005148     ucrt:api-ms-win-crt-runtime-l1-1-0.dll
 0002:00000150       __imp___acrt_iob_func      0000000180005150     ucrt:api-ms-win-crt-stdio-l1-1-0.dll
 0002:00000158       __imp_fflush               0000000180005158     ucrt:api-ms-win-crt-stdio-l1-1-0.dll
 0002:00000160       __imp___stdio_common_vsprintf 0000000180005160     ucrt:api-ms-win-crt-stdio-l1-1-0.dll
 0002:00000168       __imp___stdio_common_vfprintf 0000000180005168     ucrt:api-ms-win-crt-stdio-l1-1-0.dll
 0002:00000170       \177api-ms-win-crt-stdio-l1-1-0_NULL_THUNK_DATA 0000000180005170     ucrt:api-ms-win-crt-stdio-l1-1-0.dll
 0002:00000178       __imp__strdup              0000000180005178     ucrt:api-ms-win-crt-string-l1-1-0.dll
 0002:00000178       __imp_strdup               0000000180005178     ucrt:api-ms-win-crt-string-l1-1-0.dll
 0002:00000180       __imp_strlen               0000000180005180     ucrt:api-ms-win-crt-string-l1-1-0.dll
 0002:00000188       __imp_strncpy              0000000180005188     ucrt:api-ms-win-crt-string-l1-1-0.dll
 0002:00000190       \177api-ms-win-crt-string-l1-1-0_NULL_THUNK_DATA 0000000180005190     ucrt:api-ms-win-crt-string-l1-1-0.dll
 0002:00000198       __guard_check_icall_fptr   0000000180005198     MSVCRT:guard_support.obj
 0002:000001a0       __guard_xfg_check_icall_fptr 00000001800051a0     MSVCRT:guard_support.obj
 0002:000001a8       __guard_dispatch_icall_fptr 00000001800051a8     MSVCRT:guard_support.obj
 0002:000001b0       __guard_xfg_dispatch_icall_fptr 00000001800051b0     MSVCRT:guard_support.obj
 0002:000001b8       __guard_xfg_table_dispatch_icall_fptr 00000001800051b8     MSVCRT:guard_support.obj
 0002:000001c0       __castguard_check_failure_os_handled_fptr 00000001800051c0     MSVCRT:guard_support.obj
 0002:000001c8       __guard_memcpy_fptr        00000001800051c8     vcruntime:softmemtag.obj
 0002:000001d0       __xc_a                     00000001800051d0     MSVCRT:initializers.obj
 0002:000001d8       __xc_z                     00000001800051d8     MSVCRT:initializers.obj
 0002:000001e0       __xi_a                     00000001800051e0     MSVCRT:initializers.obj
 0002:000001f0       __xi_z                     00000001800051f0     MSVCRT:initializers.obj
 0002:000001f8       __xl_a                     00000001800051f8     MSVCRT:tlssup.obj
 0002:00000200       __xl_z                     0000000180005200     MSVCRT:tlssup.obj
 0002:00000208       __xp_a                     0000000180005208     MSVCRT:initializers.obj
 0002:00000210       __xp_z                     0000000180005210     MSVCRT:initializers.obj
 0002:00000218       __xt_a                     0000000180005218     MSVCRT:initializers.obj
 0002:00000220       __xt_z                     0000000180005220     MSVCRT:initializers.obj
 0002:00000230       g_refKindStr               0000000180005230     libStackTrace.obj
 0002:000003e0       ??_C@_09BPLDFGCI@unknown_0@ 00000001800053e0     libStackTrace.obj
 0002:000003f0       ??_C@_0BL@FPNMECJD@JVMTI_HEAP_REFERENCE_CLASS@ 00000001800053f0     libStackTrace.obj
 0002:00000410       ??_C@_0BL@FKGKKLNM@JVMTI_HEAP_REFERENCE_FIELD@ 0000000180005410     libStackTrace.obj
 0002:00000430       ??_C@_0CD@CAEHCFJF@JVMTI_HEAP_REFERENCE_ARRAY_ELEM@ 0000000180005430     libStackTrace.obj
 0002:00000458       ??_C@_0CC@DNEBMCNK@JVMTI_HEAP_REFERENCE_CLASS_LOAD@ 0000000180005458     libStackTrace.obj
 0002:00000480       ??_C@_0BN@CJMIPEBB@JVMTI_HEAP_REFERENCE_SIGNERS@ 0000000180005480     libStackTrace.obj
 0002:000004a0       ??_C@_0CH@HBOIDPEB@JVMTI_HEAP_REFERENCE_PROTECTION@ 00000001800054a0     libStackTrace.obj
 0002:000004c8       ??_C@_0BP@MDKGDGKL@JVMTI_HEAP_REFERENCE_INTERFACE@ 00000001800054c8     libStackTrace.obj
 0002:000004e8       ??_C@_0CC@JJMIHNJH@JVMTI_HEAP_REFERENCE_STATIC_FIE@ 00000001800054e8     libStackTrace.obj
 0002:00000510       ??_C@_0CD@IDHEEGID@JVMTI_HEAP_REFERENCE_CONSTANT_P@ 0000000180005510     libStackTrace.obj
 0002:00000538       ??_C@_0CA@EFFCHNG@JVMTI_HEAP_REFERENCE_SUPERCLASS@ 0000000180005538     libStackTrace.obj
 0002:00000558       ??_C@_0L@PCDFHGCJ@unknown_11@ 0000000180005558     libStackTrace.obj
 0002:00000568       ??_C@_0L@NJBICFOK@unknown_12@ 0000000180005568     libStackTrace.obj
 0002:00000578       ??_C@_0L@MAADBEKL@unknown_13@ 0000000180005578     libStackTrace.obj
 0002:00000588       ??_C@_0L@IPECICGM@unknown_14@ 0000000180005588     libStackTrace.obj
 0002:00000598       ??_C@_0L@JGFJLDCN@unknown_15@ 0000000180005598     libStackTrace.obj
 0002:000005a8       ??_C@_0L@LNHEOAOO@unknown_16@ 00000001800055a8     libStackTrace.obj
 0002:000005b8       ??_C@_0L@KEGPNBKP@unknown_17@ 00000001800055b8     libStackTrace.obj
 0002:000005c8       ??_C@_0L@CDPHMNGA@unknown_18@ 00000001800055c8     libStackTrace.obj
 0002:000005d8       ??_C@_0L@DKOMPMCB@unknown_19@ 00000001800055d8     libStackTrace.obj
 0002:000005e8       ??_C@_0L@OJGIPJDB@unknown_20@ 00000001800055e8     libStackTrace.obj
 0002:000005f8       ??_C@_0CA@KAOFNDEM@JVMTI_HEAP_REFERENCE_JNI_GLOBAL@ 00000001800055f8     libStackTrace.obj
 0002:00000618       ??_C@_0CC@HPFAJBK@JVMTI_HEAP_REFERENCE_SYSTEM_CLA@ 0000000180005618     libStackTrace.obj
 0002:00000640       ??_C@_0BN@FDEGFOHC@JVMTI_HEAP_REFERENCE_MONITOR@ 0000000180005640     libStackTrace.obj
 0002:00000660       ??_C@_0CB@HKIBCMAJ@JVMTI_HEAP_REFERENCE_STACK_LOCA@ 0000000180005660     libStackTrace.obj
 0002:00000688       ??_C@_0BP@EAACMMOE@JVMTI_HEAP_REFERENCE_JNI_LOCAL@ 0000000180005688     libStackTrace.obj
 0002:000006a8       ??_C@_0BM@IJDEOGOE@JVMTI_HEAP_REFERENCE_THREAD@ 00000001800056a8     libStackTrace.obj
 0002:000006c8       ??_C@_0BL@EDGPPKC@JVMTI_HEAP_REFERENCE_OTHER@ 00000001800056c8     libStackTrace.obj
 0002:000006e4       ??_C@_04BCJPDBDA@Code@     00000001800056e4     libStackTrace.obj
 0002:000006f0       ??_C@_0BA@OCLMCFKC@LineNumberTable@ 00000001800056f0     libStackTrace.obj
 0002:00000700       ??_C@_0BD@CPAEPILC@LocalVariableTable@ 0000000180005700     libStackTrace.obj
 0002:00000718       ??_C@_0BH@NMBDNHBD@LocalVariableTypeTable@ 0000000180005718     libStackTrace.obj
 0002:00000730       ??_C@_0O@HIHEEDNJ@StackMapTable@ 0000000180005730     libStackTrace.obj
 0002:00000740       ??_C@_0L@HCDIAMJG@?9?5?$CFs?0?5?$CFd?3?5@ 0000000180005740     libStackTrace.obj
 0002:00000750       ??_C@_0JI@HLPECLFI@?$CD?5?4?4?4?6?$CD?5ERROR?3?5too?5many?5complai@ 0000000180005750     libStackTrace.obj
 0002:000007f0       ??_C@_0ED@JNEKCCOB@The?5following?5fake?5exception?5st@ 00000001800057f0     libStackTrace.obj
 0002:00000838       ??_C@_0CN@FCNMDFBH@nsk?4share?4Fake_Exception_for_RU@ 0000000180005838     libStackTrace.obj
 0002:00000868       ??_C@_08PGFFNAEI@?$CI?$CFs?3?$CFd?$CJ?5@ 0000000180005868     libStackTrace.obj
 0002:00000878       ??_C@_0DP@IENMAEGI@s?2test?2hotspot?2jtreg?2vmTestbase@ 0000000180005878     libStackTrace.obj
 0002:000008b8       ??_C@_0BL@NDJLFFJB@?7at?5nsk_lvcomplain?$CI?$CFs?3?$CFd?$CJ?6@ 00000001800058b8     libStackTrace.obj
 0002:000008d8       ??_C@_0BC@JOOKAFKF@?$CD?5ERROR?3?5?$CFs?0?5?$CFd?3?5@ 00000001800058d8     libStackTrace.obj
 0002:000008f0       ??_C@_09KJEAHMEH@?$CD?5ERROR?3?5@ 00000001800058f0     libStackTrace.obj
 0002:000008fc       ??_C@_02GPIOPFAK@?$DO?$DO@ 00000001800058fc     libStackTrace.obj
 0002:00000900       ??_C@_02FODMEDOG@?$DM?$DM@ 0000000180005900     libStackTrace.obj
 0002:00000904       ??_C@_02DJGKEECL@?4?4@     0000000180005904     libStackTrace.obj
 0002:00000908       ??_C@_0O@CJPGJOAF@?9?5?$CFs?0?5?$CFd?3?5?$CFs?5@ 0000000180005908     libStackTrace.obj
 0002:00000918       ??_C@_0CB@IAKPDOIC@?$CD?5?5?5verified?5assertion?5is?5FALSE@ 0000000180005918     libStackTrace.obj
 0002:00000940       ??_C@_0CO@LGONDEPD@stdout?3?5fflush?5failed?5?9?5err?$DN?$CFd?5@ 0000000180005940     libStackTrace.obj
 0002:00000970       ??_C@_0CO@KBGKJPBD@stderr?3?5fflush?5failed?5?9?5err?$DN?$CFd?5@ 0000000180005970     libStackTrace.obj
 0002:000009a0       ??_C@_0BB@JCNMKLLK@JVMTI_ERROR_NONE@ 00000001800059a0     libStackTrace.obj
 0002:000009b8       ??_C@_0BL@LDIMKLPH@JVMTI_ERROR_INVALID_THREAD@ 00000001800059b8     libStackTrace.obj
 0002:000009d8       ??_C@_0CB@PJFPAIKJ@JVMTI_ERROR_INVALID_THREAD_GROU@ 00000001800059d8     libStackTrace.obj
 0002:00000a00       ??_C@_0BN@LLMKHMNF@JVMTI_ERROR_INVALID_PRIORITY@ 0000000180005a00     libStackTrace.obj
 0002:00000a20       ??_C@_0CB@MBOFKAGB@JVMTI_ERROR_THREAD_NOT_SUSPENDE@ 0000000180005a20     libStackTrace.obj
 0002:00000a48       ??_C@_0BN@FABOLPBI@JVMTI_ERROR_THREAD_SUSPENDED@ 0000000180005a48     libStackTrace.obj
 0002:00000a68       ??_C@_0BN@FDGNOBJM@JVMTI_ERROR_THREAD_NOT_ALIVE@ 0000000180005a68     libStackTrace.obj
 0002:00000a88       ??_C@_0BL@GOBIFKNJ@JVMTI_ERROR_INVALID_OBJECT@ 0000000180005a88     libStackTrace.obj
 0002:00000aa8       ??_C@_0BK@FCMAJPPC@JVMTI_ERROR_INVALID_CLASS@ 0000000180005aa8     libStackTrace.obj
 0002:00000ac8       ??_C@_0BP@IKLLBKEB@JVMTI_ERROR_CLASS_NOT_PREPARED@ 0000000180005ac8     libStackTrace.obj
 0002:00000ae8       ??_C@_0BN@KLPPLKG@JVMTI_ERROR_INVALID_METHODID@ 0000000180005ae8     libStackTrace.obj
 0002:00000b08       ??_C@_0BN@BCEKOKND@JVMTI_ERROR_INVALID_LOCATION@ 0000000180005b08     libStackTrace.obj
 0002:00000b28       ??_C@_0BM@DFDGPME@JVMTI_ERROR_INVALID_FIELDID@ 0000000180005b28     libStackTrace.obj
 0002:00000b48       ??_C@_0BL@NELIEPEC@JVMTI_ERROR_NO_MORE_FRAMES@ 0000000180005b48     libStackTrace.obj
 0002:00000b68       ??_C@_0BJ@BDBECFDM@JVMTI_ERROR_OPAQUE_FRAME@ 0000000180005b68     libStackTrace.obj
 0002:00000b88       ??_C@_0BK@MIIFNLOB@JVMTI_ERROR_TYPE_MISMATCH@ 0000000180005b88     libStackTrace.obj
 0002:00000ba8       ??_C@_0BJ@HPCAOILC@JVMTI_ERROR_INVALID_SLOT@ 0000000180005ba8     libStackTrace.obj
 0002:00000bc8       ??_C@_0BG@CHILOPNI@JVMTI_ERROR_DUPLICATE@ 0000000180005bc8     libStackTrace.obj
 0002:00000be0       ??_C@_0BG@DIEMLHKM@JVMTI_ERROR_NOT_FOUND@ 0000000180005be0     libStackTrace.obj
 0002:00000bf8       ??_C@_0BM@NHMCKHOB@JVMTI_ERROR_INVALID_MONITOR@ 0000000180005bf8     libStackTrace.obj
 0002:00000c18       ??_C@_0BO@PPEDAJGL@JVMTI_ERROR_NOT_MONITOR_OWNER@ 0000000180005c18     libStackTrace.obj
 0002:00000c38       ??_C@_0BG@FCAIPEID@JVMTI_ERROR_INTERRUPT@ 0000000180005c38     libStackTrace.obj
 0002:00000c50       ??_C@_0CB@EGDBNKOI@JVMTI_ERROR_INVALID_CLASS_FORMA@ 0000000180005c50     libStackTrace.obj
 0002:00000c78       ??_C@_0CG@DGKOGIAL@JVMTI_ERROR_CIRCULAR_CLASS_DEFI@ 0000000180005c78     libStackTrace.obj
 0002:00000ca0       ??_C@_0BP@ICEALPKC@JVMTI_ERROR_FAILS_VERIFICATION@ 0000000180005ca0     libStackTrace.obj
 0002:00000cc0       ??_C@_0DC@JDACLMIO@JVMTI_ERROR_UNSUPPORTED_REDEFIN@ 0000000180005cc0     libStackTrace.obj
 0002:00000cf8       ??_C@_0DE@GKDKNOMJ@JVMTI_ERROR_UNSUPPORTED_REDEFIN@ 0000000180005cf8     libStackTrace.obj
 0002:00000d30       ??_C@_0BO@LAFKIOG@JVMTI_ERROR_INVALID_TYPESTATE@ 0000000180005d30     libStackTrace.obj
 0002:00000d50       ??_C@_0DH@INDGCLLB@JVMTI_ERROR_UNSUPPORTED_REDEFIN@ 0000000180005d50     libStackTrace.obj
 0002:00000d88       ??_C@_0DE@NHEOMMGI@JVMTI_ERROR_UNSUPPORTED_REDEFIN@ 0000000180005d88     libStackTrace.obj
 0002:00000dc0       ??_C@_0CA@EKPNJOEP@JVMTI_ERROR_UNSUPPORTED_VERSION@ 0000000180005dc0     libStackTrace.obj
 0002:00000de0       ??_C@_0BN@OFFMAHHL@JVMTI_ERROR_NAMES_DONT_MATCH@ 0000000180005de0     libStackTrace.obj
 0002:00000e00       ??_C@_0DN@HHBBLAKE@JVMTI_ERROR_UNSUPPORTED_REDEFIN@ 0000000180005e00     libStackTrace.obj
 0002:00000e40       ??_C@_0DO@HMBGBGNA@JVMTI_ERROR_UNSUPPORTED_REDEFIN@ 0000000180005e40     libStackTrace.obj
 0002:00000e80       ??_C@_0BP@PBECGKHJ@JVMTI_ERROR_UNMODIFIABLE_CLASS@ 0000000180005e80     libStackTrace.obj
 0002:00000ea0       ??_C@_0BK@CANILEHF@JVMTI_ERROR_NOT_AVAILABLE@ 0000000180005ea0     libStackTrace.obj
 0002:00000ec0       ??_C@_0CE@INJKMEFK@JVMTI_ERROR_MUST_POSSESS_CAPABI@ 0000000180005ec0     libStackTrace.obj
 0002:00000ee8       ??_C@_0BJ@LBFPFPDM@JVMTI_ERROR_NULL_POINTER@ 0000000180005ee8     libStackTrace.obj
 0002:00000f08       ??_C@_0BP@CHJPNNEM@JVMTI_ERROR_ABSENT_INFORMATION@ 0000000180005f08     libStackTrace.obj
 0002:00000f28       ??_C@_0BP@OMFMNLC@JVMTI_ERROR_INVALID_EVENT_TYPE@ 0000000180005f28     libStackTrace.obj
 0002:00000f48       ??_C@_0BN@BIBNPHHO@JVMTI_ERROR_ILLEGAL_ARGUMENT@ 0000000180005f48     libStackTrace.obj
 0002:00000f68       ??_C@_0BK@KKNDHDCE@JVMTI_ERROR_NATIVE_METHOD@ 0000000180005f68     libStackTrace.obj
 0002:00000f88       ??_C@_0BK@PMKCFHAE@JVMTI_ERROR_OUT_OF_MEMORY@ 0000000180005f88     libStackTrace.obj
 0002:00000fa8       ??_C@_0BK@NNJBDMNB@JVMTI_ERROR_ACCESS_DENIED@ 0000000180005fa8     libStackTrace.obj
 0002:00000fc8       ??_C@_0BI@GHECLMNC@JVMTI_ERROR_WRONG_PHASE@ 0000000180005fc8     libStackTrace.obj
 0002:00000fe0       ??_C@_0BF@OLIHJOII@JVMTI_ERROR_INTERNAL@ 0000000180005fe0     libStackTrace.obj
 0002:00000ff8       ??_C@_0BO@EOHGKJHI@JVMTI_ERROR_UNATTACHED_THREAD@ 0000000180005ff8     libStackTrace.obj
 0002:00001018       ??_C@_0CA@LKHFDACL@JVMTI_ERROR_INVALID_ENVIRONMENT@ 0000000180006018     libStackTrace.obj
 0002:00001038       ??_C@_0BA@MMFHLOKK@?$DMunknown?5error?$DO@ 0000000180006038     libStackTrace.obj
 0002:00001048       ??_C@_0CF@CBHOKDB@throwable?5?$DN?5jni?9?$DOExceptionOccur@ 0000000180006048     libStackTrace.obj
 0002:00001070       ??_C@_03OFAPEBGM@?$CFs?6@  0000000180006070     libStackTrace.obj
 0002:00001078       ??_C@_0DM@LPIGEGNJ@s?2test?2hotspot?2jtreg?2vmTestbase@ 0000000180006078     libStackTrace.obj
 0002:000010b8       ??_C@_0CC@NFCNPEPK@Exception?5in?5JNI?5call?5?$CIcleared?$CJ@ 00000001800060b8     libStackTrace.obj
 0002:000010e0       ??_C@_0BJ@IBAKFIKF@jni?9?$DOExceptionDescribe?$CI?$CJ@ 00000001800060e0     libStackTrace.obj
 0002:00001100       ??_C@_0BG@GGKALKMH@jni?9?$DOExceptionClear?$CI?$CJ@ 0000000180006100     libStackTrace.obj
 0002:00001118       ??_C@_0CF@JMGFGJLJ@?$CD?5?5?5verified?5JNI?5assertion?5is?5F@ 0000000180006118     libStackTrace.obj
 0002:00001140       ??_C@_0CB@MLNJNCLJ@?5?5jvmti?5error?3?5code?$DN?$CFd?0?5name?$DN?$CFs@ 0000000180006140     libStackTrace.obj
 0002:00001168       ??_C@_0CD@OHBGDKMK@?$CD?5?5?5jvmti?5error?3?5code?$DN?$CFd?0?5name?$DN@ 0000000180006168     libStackTrace.obj
 0002:00001190       ??_C@_0CG@JNNCGPHB@?$CD?5?5?5error?5expected?3?5code?$DN?$CFd?0?5na@ 0000000180006190     libStackTrace.obj
 0002:000011c0       ??_C@_0EB@IMGKPCGE@?$CIstr_obj?5?$DN?5jni?9?$DONewStringUTF?$CIco@ 00000001800061c0     libStackTrace.obj
 0002:00001210       ??_C@_0EA@HFOGGBCC@s?2test?2hotspot?2jtreg?2vmTestbase@ 0000000180006210     libStackTrace.obj
 0002:00001250       ??_C@_05KKCIMGE@error@     0000000180006250     libStackTrace.obj
 0002:00001258       ??_C@_0CJ@JACLEAA@Test?5failed?5by?5setFailStatus?$CI?$CJ?4@ 0000000180006258     libStackTrace.obj
 0002:00001290       ??_C@_0EA@PNBCDMOA@s?2test?2hotspot?2jtreg?2vmTestbase@ 0000000180006290     libStackTrace.obj
 0002:000012d0       ??_C@_0DI@ILAHDLMP@?$CI?$CKagentThreadProc?$CJ?$CIjvmti_env?0?5a@ 00000001800062d0     libStackTrace.obj
 0002:00001308       ??_C@_0BD@KDBALNLB@JVMTI?5agent?5thread@ 0000000180006308     libStackTrace.obj
 0002:00001320       ??_C@_0BB@NOKBFPFO@java?1lang?1Thread@ 0000000180006320     libStackTrace.obj
 0002:00001334       ??_C@_06FALKBLGB@?$DMinit?$DO@ 0000000180006334     libStackTrace.obj
 0002:00001340       ??_C@_0BG@IKDDPPGD@?$CILjava?1lang?1String?$DL?$CJV@ 0000000180006340     libStackTrace.obj
 0002:00001360       ??_C@_0EB@IFJBFEKC@?$CIthreadClass?5?$DN?5jni_env?9?$DOFindCla@ 0000000180006360     libStackTrace.obj
 0002:000013b0       ??_C@_0GF@FGFIBKKL@?$CIthreadCtor?5?$DN?5jni_env?9?$DOGetMetho@ 00000001800063b0     libStackTrace.obj
 0002:00001418       ??_C@_0DN@NCPDJLOG@?$CIthreadName?5?$DN?5jni_env?9?$DONewStrin@ 0000000180006418     libStackTrace.obj
 0002:00001460       ??_C@_0FE@PFKODBGC@?$CIthreadObject?5?$DN?5jni_env?9?$DONewObj@ 0000000180006460     libStackTrace.obj
 0002:000014c0       ??_C@_0ED@HOBAHHJI@?$CIthreadGlobalRef?5?$DN?5jni_env?9?$DONew@ 00000001800064c0     libStackTrace.obj
 0002:00001510       ??_C@_0FN@HNJJAHFC@jvmti_env?9?$DORunAgentThread?$CIagent@ 0000000180006510     libStackTrace.obj
 0002:00001570       ??_C@_0EA@MOJDNKDF@Debuggee?5status?5sync?5aborted?5be@ 0000000180006570     libStackTrace.obj
 0002:000015b0       ??_C@_0EA@EEOEJAEN@status?5?$DN?5syncDebuggeeStatus?$CIjni@ 00000001800065b0     libStackTrace.obj
 0002:000015f0       ??_C@_0BL@JBCFNBMB@nsk_jvmti_resetAgentData?$CI?$CJ@ 00000001800065f0     libStackTrace.obj
 0002:00001610       ??_C@_0EL@LPBEELIP@s?2test?2hotspot?2jtreg?2vmTestbase@ 0000000180006610     libStackTrace.obj
 0002:00001660       ??_C@_0CK@JDAMFDMJ@jvmti?9?$DOSetTag?$CIo?0?5tag?$CJ?5?$DN?$DN?5JVMTI_@ 0000000180006660     libStackTrace.obj
 0002:00001690       ??_C@_0CC@DAMNHKNI@Can?8t?5set?5tag?5?$CFli?5for?5object?5?$CFl@ 0000000180006690     libStackTrace.obj
 0002:000016b8       ??_C@_0DL@HAJPNKEF@jvmti?9?$DOGetObjectHashCode?$CIo?0?5?$CGha@ 00000001800066b8     libStackTrace.obj
 0002:000016f8       ??_C@_0BL@JFPIEOBF@Can?8t?5get?5hash?5object?5?$CFlx?6@ 00000001800066f8     libStackTrace.obj
 0002:00001718       ??_C@_0BG@DICPHBKN@setTag?3?5?$CF08x?5?$DM?9?5?$CF?53li@ 0000000180006718     libStackTrace.obj
 0002:00001730       ??_C@_0DH@FCEEBDMJ@?$CIs?5?$DN?5jni?9?$DOGetStringUTFChars?$CIsIn@ 0000000180006730     libStackTrace.obj
 0002:00001768       ??_C@_0BJ@OKKGHDCN@Can?8t?5get?5string?5at?5?$CF?$CDp?6@ 0000000180006768     libStackTrace.obj
 0002:00001788       ??_C@_0BP@EKFLGGFJ@Can?8t?5get?5string?5at?5?$CF?$CDp?3?5null?6@ 0000000180006788     libStackTrace.obj
 0002:000017a8       ??_C@_06ICODBHCL@?5?1?1?5?$CFs@ 00000001800067a8     libStackTrace.obj
 0002:000017b0       ??_C@_0DB@KGFPLEGO@?$CIr?5?$DN?5jvmti?9?$DOGetTag?$CIo?0?5?$CGtag?$CJ?$CJ?5?$DN?$DN@ 00000001800067b0     libStackTrace.obj
 0002:000017e8       ??_C@_0CO@PDAGBCGJ@Can?8t?5GetTag?5for?5object?5?$CFlx?4?5Re@ 00000001800067e8     libStackTrace.obj
 0002:00001818       ??_C@_0CH@HPEODOHC@TEST_BUG?3?5Max?4?5number?5of?5refs?5r@ 0000000180006818     libStackTrace.obj
 0002:00001840       ??_C@_0DI@PHFCABIM@?$CIr?5?$DN?5jvmti?9?$DOGetTag?$CIfrom?0?5?$CGtagFr@ 0000000180006840     libStackTrace.obj
 0002:00001878       ??_C@_0DI@MDEGFNKD@TEST_BUG?3?5Can?8t?5GetTag?5for?5obje@ 0000000180006878     libStackTrace.obj
 0002:000018b0       ??_C@_0DE@MLELJAHM@?$CIr?5?$DN?5jvmti?9?$DOGetTag?$CIto?0?5?$CGtagTo?$CJ?$CJ@ 00000001800068b0     libStackTrace.obj
 0002:000018e8       ??_C@_09OPJEJKBL@printdump@ 00000001800068e8     libStackTrace.obj
 0002:000018f8       ??_C@_0CJ@KCDEKOCJ@Wrong?5result?5of?5a?5valid?5call?5to@ 00000001800068f8     libStackTrace.obj
 0002:00001928       ??_C@_0CI@EDEMEGFA@GetPotentialCapabilities?5return@ 0000000180006928     libStackTrace.obj
 0002:00001950       ??_C@_03PMGGPEJJ@?$CFd?6@  0000000180006950     libStackTrace.obj
 0002:00001958       ??_C@_0O@IEOHCAJP@Rawmonitor?9?$CFd@ 0000000180006958     libStackTrace.obj
 0002:00001968       ??_C@_0BL@PPNDBPKK@jvmti?5create?5raw?5monitor?5?6@ 0000000180006968     libStackTrace.obj
 0002:00001988       ??_C@_0CD@FAOAJHGL@Error?3?5ForceGarbageCollection?5?$CF@ 0000000180006988     libStackTrace.obj
 0002:000019b0       ??_C@_0BK@KEFLCGDC@jvmti?5Raw?5monitor?5enter?5?6@ 00000001800069b0     libStackTrace.obj
 0002:000019d0       ??_C@_0BO@OJFPHDDP@Error?3?5Raw?5monitor?5enter?5?$CFd?5?6@ 00000001800069d0     libStackTrace.obj
 0002:000019f0       ??_C@_0BJ@OJLKHENF@jvmti?5raw?5monitor?5exit?5?6@ 00000001800069f0     libStackTrace.obj
 0002:00001a10       ??_C@_0BL@GKGBEHOI@Error?3?5RawMonitorExit?5?$CFd?5?6@ 0000000180006a10     libStackTrace.obj
 0002:00001a30       ??_C@_0BH@PILJFGHG@jvmti?5RawMonitorWait?5?6@ 0000000180006a30     libStackTrace.obj
 0002:00001a48       ??_C@_0BL@EJFJOCBH@Error?3?5RawMonitorWait?5?$CFd?5?6@ 0000000180006a48     libStackTrace.obj
 0002:00001a68       ??_C@_0BJ@DLFONEKK@jvmti?5RawMonitorNotify?5?6@ 0000000180006a68     libStackTrace.obj
 0002:00001a88       ??_C@_0BN@EJGKLMHH@Error?3?5RawMonitorNotify?5?$CFd?5?6@ 0000000180006a88     libStackTrace.obj
 0002:00001aa8       ??_C@_0BG@MDNBHIDB@jvmti?5GetFrameCount?5?6@ 0000000180006aa8     libStackTrace.obj
 0002:00001ac0       ??_C@_0CE@CMHEGKH@Error?3?5GetFrameCount?5returned?5?5@ 0000000180006ac0     libStackTrace.obj
 0002:00001ae8       ??_C@_0BG@KLMKFCMD@jvmti?5GetStackTrace?5?6@ 0000000180006ae8     libStackTrace.obj
 0002:00001b00       ??_C@_0CC@LBLLBNPM@Error?3?5Allocate?5failed?5with?5?5?$CFd@ 0000000180006b00     libStackTrace.obj
 0002:00001b28       ??_C@_0CH@MFGAKIOD@Error?3?5SuspendThread?5failed?5wit@ 0000000180006b28     libStackTrace.obj
 0002:00001b50       ??_C@_0BK@FMLENDOH@Error?3?5GetStackTrace?5?$CFd?5?6@ 0000000180006b50     libStackTrace.obj
 0002:00001b70       ??_C@_0BL@CAGOEKHD@Error?3?5GetStackTrace2?5?$CFd?5?6@ 0000000180006b70     libStackTrace.obj
 0002:00001b90       ??_C@_0DE@NFCMJPJA@Error?3?5mismatch?5res_count?5?$DN?5?$CFd?0@ 0000000180006b90     libStackTrace.obj
 0002:00001bc8       ??_C@_0BF@CDFMEDPJ@Error?3?5wrong?5method?6@ 0000000180006bc8     libStackTrace.obj
 0002:00001be0       ??_C@_0CI@ILFKNPNA@Error?3?5mismatch?5res_count?5?$DN?5?$CFd?0@ 0000000180006be0     libStackTrace.obj
 0002:00001c08       ??_C@_0BJ@EJNKHAEN@Error?3?5wrong?5neg?5method?6@ 0000000180006c08     libStackTrace.obj
 0002:00001c28       ??_C@_0M@DIGFGDHP@Count?5?$DN?5?$CFd?6@ 0000000180006c28     libStackTrace.obj
 0002:00001c38       ??_C@_0CG@EHEDMDLG@Error?3?5ResumeThread?5failed?5with@ 0000000180006c38     libStackTrace.obj
 0002:00001c60       ??_C@_0BH@LKBPMHHF@?5Java?5Stack?5trace?5?9?9?9?6@ 0000000180006c60     libStackTrace.obj
 0002:00001c78       ??_C@_0CF@HPJKBGDC@Error?3?5GetMethodDeclaringClass?5@ 0000000180006c78     libStackTrace.obj
 0002:00001ca0       ??_C@_0BP@LFIKIAMN@Error?3?5GetClassSignature?5?$CFd?5?5?6@ 0000000180006ca0     libStackTrace.obj
 0002:00001cc0       ??_C@_0BL@OJMCGCKC@Error?3?5GetMethodName?5?$CFd?5?5?6@ 0000000180006cc0     libStackTrace.obj
 0002:00001ce0       ??_C@_0BL@OEOPAHNI@?$FL?$CFd?$FN?5?5?$CFs?3?3?$CFs?$CI?$CFs?$CJ?5at?5?$CFlld?5?6@ 0000000180006ce0     libStackTrace.obj
 0002:00001d00       ??_C@_0CE@LGABKEJM@Error?3?5Deallocate?5failed?5with?5?5@ 0000000180006d00     libStackTrace.obj
 0002:00001d40       ??_C@_1EC@JIJBPKFM@?$AAa?$AAp?$AAi?$AA?9?$AAm?$AAs?$AA?9?$AAw?$AAi?$AAn?$AA?9?$AAc?$AAo?$AAr?$AAe@ 0000000180006d40     MSVCRT:thread_safe_statics.obj
 0002:00001d88       ??_C@_1BK@MGMFAEKH@?$AAk?$AAe?$AAr?$AAn?$AAe?$AAl?$AA3?$AA2?$AA?4?$AAd?$AAl?$AAl@ 0000000180006d88     MSVCRT:thread_safe_statics.obj
 0002:00001da8       ??_C@_0BJ@JEBJOJFJ@SleepConditionVariableCS@ 0000000180006da8     MSVCRT:thread_safe_statics.obj
 0002:00001dc8       ??_C@_0BJ@PGPPEPCC@WakeAllConditionVariable@ 0000000180006dc8     MSVCRT:thread_safe_statics.obj
 0002:00001de8       _pDefaultRawDllMain        0000000180006de8     MSVCRT:dll_dllmain.obj
 0002:00001de8       _pRawDllMain               0000000180006de8     MSVCRT:dll_dllmain.obj
 0002:00001df0       __xmm@ffffffffffffffffffffffffffffffff 0000000180006df0     MSVCRT:utility.obj
 0002:00001e00       _load_config_used          0000000180006e00     MSVCRT:loadcfg.obj
 0002:00002000       _tls_used                  0000000180007000     MSVCRT:tlssup.obj
 0002:00002028       __volatile_metadata        0000000180007028     <linker-defined>
 0002:000023e8       __rtc_iaa                  00000001800073e8     MSVCRT:initsect.obj
 0002:000023f0       __rtc_izz                  00000001800073f0     MSVCRT:initsect.obj
 0002:000023f8       __rtc_taa                  00000001800073f8     MSVCRT:initsect.obj
 0002:00002400       __rtc_tzz                  0000000180007400     MSVCRT:initsect.obj
 0002:00002408       _tls_start                 0000000180007408     MSVCRT:tlssup.obj
 0002:0000240c       _Init_thread_epoch         000000018000740c     MSVCRT:thread_safe_statics.obj
 0002:00002410       _tls_end                   0000000180007410     MSVCRT:tlssup.obj
 0002:00002ce4       __IMPORT_DESCRIPTOR_KERNEL32 0000000180007ce4     kernel32:KERNEL32.dll
 0002:00002cf8       __IMPORT_DESCRIPTOR_VCRUNTIME140 0000000180007cf8     vcruntime:VCRUNTIME140.dll
 0002:00002d0c       __IMPORT_DESCRIPTOR_api-ms-win-crt-runtime-l1-1-0 0000000180007d0c     ucrt:api-ms-win-crt-runtime-l1-1-0.dll
 0002:00002d20       __IMPORT_DESCRIPTOR_api-ms-win-crt-stdio-l1-1-0 0000000180007d20     ucrt:api-ms-win-crt-stdio-l1-1-0.dll
 0002:00002d34       __IMPORT_DESCRIPTOR_api-ms-win-crt-string-l1-1-0 0000000180007d34     ucrt:api-ms-win-crt-string-l1-1-0.dll
 0002:00002d48       __NULL_IMPORT_DESCRIPTOR   0000000180007d48     kernel32:KERNEL32.dll
 0003:00000030       _Init_global_epoch         0000000180009030     MSVCRT:thread_safe_statics.obj
 0003:00000040       __security_cookie          0000000180009040     MSVCRT:gs_cookie.obj
 0003:00000048       __security_cookie_complement 0000000180009048     MSVCRT:gs_cookie.obj
 0003:00000050       __scrt_native_dllmain_reason 0000000180009050     MSVCRT:utility.obj
 0003:00000058       __isa_available            0000000180009058     MSVCRT:cpu_disp.obj
 0003:0000005c       __isa_enabled              000000018000905c     MSVCRT:cpu_disp.obj
 0003:00000060       __memset_fast_string_threshold 0000000180009060     MSVCRT:cpu_disp.obj
 0003:00000068       __memset_nt_threshold      0000000180009068     MSVCRT:cpu_disp.obj
 0003:00000070       __scrt_ucrt_dll_is_in_use  0000000180009070     MSVCRT:ucrt_stubs.obj
 0003:00000080       g_wrongHeapCallbacks       0000000180009080     libStackTrace.obj
 0003:00000100       g_szTagInfo                0000000180009100     libStackTrace.obj
 0003:00002040       g_tagFlags                 000000018000b040     libStackTrace.obj
 0003:00002428       g_refsToVerifyCnt          000000018000b428     libStackTrace.obj
 0003:0000242c       g_fakeUserData             000000018000b42c     libStackTrace.obj
 0003:00002430       g_tagVisitCount            000000018000b430     libStackTrace.obj
 0003:000033d0       g_refsToVerify             000000018000c3d0     libStackTrace.obj
 0003:0001aad0       g_userDataError            0000000180023ad0     libStackTrace.obj
 0003:0001aad4       iGlobalStatus              0000000180023ad4     libStackTrace.obj
 0003:0001aad8       jvmti                      0000000180023ad8     libStackTrace.obj
 0003:0001aae0       susp_thrd                  0000000180023ae0     libStackTrace.obj
 0003:0001e960       jraw_monitor               0000000180027960     libStackTrace.obj
 0003:0001ea00       process_once               0000000180027a00     libStackTrace.obj
 0003:0001ea04       printdump                  0000000180027a04     libStackTrace.obj
 0003:0001eba8       ?_OptionsStorage@?1??__local_stdio_printf_options@@9@4_KA 0000000180027ba8     libStackTrace.obj
 0003:0001f168       _tls_index                 0000000180028168     MSVCRT:tlssup.obj
 0003:0001f170       __scrt_current_native_startup_state 0000000180028170     MSVCRT:utility.obj
 0003:0001f178       __scrt_native_startup_lock 0000000180028178     MSVCRT:utility.obj
 0003:0001f1b8       __scrt_debugger_hook_flag  00000001800281b8     MSVCRT:utility_desktop.obj
 0003:0001f1c0       ?__type_info_root_node@@3U__type_info_node@@A 00000001800281c0     MSVCRT:tncleanup.obj
 0003:0001f1d0       ?_OptionsStorage@?1??__local_stdio_scanf_options@@9@4_KA 00000001800281d0     MSVCRT:default_local_stdio_options.obj
 0003:0001f1d8       __favor                    00000001800281d8     MSVCRT:cpu_disp.obj
 0003:0001f1e0       __dyn_tls_init_callback    00000001800281e0     <common>

 entry point at        0001:000028b0

 Static symbols

 0000:fffd5000       .debug$S                   0000000180000000     StackTrace.exp
 0000:fffd5000       .debug$S                   0000000180000000     vcruntime:VCRUNTIME140.dll
 0000:fffd5000       .debug$S                   0000000180000000     vcruntime:VCRUNTIME140.dll
 0000:fffd5000       .debug$S                   0000000180000000     vcruntime:VCRUNTIME140.dll
 0000:fffd5000       .debug$S                   0000000180000000     vcruntime:VCRUNTIME140.dll
 0000:fffd5000       .debug$S                   0000000180000000     vcruntime:VCRUNTIME140.dll
 0000:fffd5000       .debug$S                   0000000180000000     vcruntime:VCRUNTIME140.dll
 0000:fffd5000       .debug$S                   0000000180000000     vcruntime:VCRUNTIME140.dll
 0000:fffd5000       .debug$S                   0000000180000000     vcruntime:VCRUNTIME140.dll
 0000:fffd5000       .debug$S                   0000000180000000     ucrt:api-ms-win-crt-convert-l1-1-0.dll
 0002:ffffb000       .idata$6                   0000000180000000     ucrt:api-ms-win-crt-convert-l1-1-0.dll
 0000:fffd5000       .debug$S                   0000000180000000     ucrt:api-ms-win-crt-heap-l1-1-0.dll
 0000:fffd5000       .debug$S                   0000000180000000     ucrt:api-ms-win-crt-heap-l1-1-0.dll
 0000:fffd5000       .debug$S                   0000000180000000     ucrt:api-ms-win-crt-heap-l1-1-0.dll
 0000:fffd5000       .debug$S                   0000000180000000     ucrt:api-ms-win-crt-heap-l1-1-0.dll
 0002:ffffb000       .idata$6                   0000000180000000     ucrt:api-ms-win-crt-heap-l1-1-0.dll
 0000:fffd5000       .debug$S                   0000000180000000     ucrt:api-ms-win-crt-runtime-l1-1-0.dll
 0000:fffd5000       .debug$S                   0000000180000000     ucrt:api-ms-win-crt-runtime-l1-1-0.dll
 0000:fffd5000       .debug$S                   0000000180000000     ucrt:api-ms-win-crt-runtime-l1-1-0.dll
 0000:fffd5000       .debug$S                   0000000180000000     ucrt:api-ms-win-crt-runtime-l1-1-0.dll
 0000:fffd5000       .debug$S                   0000000180000000     ucrt:api-ms-win-crt-runtime-l1-1-0.dll
 0000:fffd5000       .debug$S                   0000000180000000     ucrt:api-ms-win-crt-runtime-l1-1-0.dll
 0000:fffd5000       .debug$S                   0000000180000000     ucrt:api-ms-win-crt-runtime-l1-1-0.dll
 0000:fffd5000       .debug$S                   0000000180000000     ucrt:api-ms-win-crt-runtime-l1-1-0.dll
 0000:fffd5000       .debug$S                   0000000180000000     ucrt:api-ms-win-crt-runtime-l1-1-0.dll
 0000:fffd5000       .debug$S                   0000000180000000     ucrt:api-ms-win-crt-runtime-l1-1-0.dll
 0000:fffd5000       .debug$S                   0000000180000000     ucrt:api-ms-win-crt-runtime-l1-1-0.dll
 0000:fffd5000       .debug$S                   0000000180000000     ucrt:api-ms-win-crt-runtime-l1-1-0.dll
 0000:fffd5000       .debug$S                   0000000180000000     ucrt:api-ms-win-crt-runtime-l1-1-0.dll
 0000:fffd5000       .debug$S                   0000000180000000     ucrt:api-ms-win-crt-runtime-l1-1-0.dll
 0000:fffd5000       .debug$S                   0000000180000000     ucrt:api-ms-win-crt-runtime-l1-1-0.dll
 0000:fffd5000       .debug$S                   0000000180000000     ucrt:api-ms-win-crt-runtime-l1-1-0.dll
 0000:fffd5000       .debug$S                   0000000180000000     ucrt:api-ms-win-crt-stdio-l1-1-0.dll
 0000:fffd5000       .debug$S                   0000000180000000     ucrt:api-ms-win-crt-stdio-l1-1-0.dll
 0000:fffd5000       .debug$S                   0000000180000000     ucrt:api-ms-win-crt-stdio-l1-1-0.dll
 0000:fffd5000       .debug$S                   0000000180000000     ucrt:api-ms-win-crt-stdio-l1-1-0.dll
 0000:fffd5000       .debug$S                   0000000180000000     ucrt:api-ms-win-crt-stdio-l1-1-0.dll
 0000:fffd5000       .debug$S                   0000000180000000     ucrt:api-ms-win-crt-stdio-l1-1-0.dll
 0000:fffd5000       .debug$S                   0000000180000000     ucrt:api-ms-win-crt-stdio-l1-1-0.dll
 0000:fffd5000       .debug$S                   0000000180000000     ucrt:api-ms-win-crt-stdio-l1-1-0.dll
 0000:fffd5000       .debug$S                   0000000180000000     ucrt:api-ms-win-crt-stdio-l1-1-0.dll
 0000:fffd5000       .debug$S                   0000000180000000     ucrt:api-ms-win-crt-stdio-l1-1-0.dll
 0000:fffd5000       .debug$S                   0000000180000000     ucrt:api-ms-win-crt-string-l1-1-0.dll
 0000:fffd5000       .debug$S                   0000000180000000     ucrt:api-ms-win-crt-string-l1-1-0.dll
 0000:fffd5000       .debug$S                   0000000180000000     ucrt:api-ms-win-crt-string-l1-1-0.dll
 0000:fffd5000       .debug$S                   0000000180000000     ucrt:api-ms-win-crt-string-l1-1-0.dll
 0000:fffd5000       .debug$S                   0000000180000000     ucrt:api-ms-win-crt-string-l1-1-0.dll
 0000:fffd5000       .debug$S                   0000000180000000     ucrt:api-ms-win-crt-string-l1-1-0.dll
 0000:fffd5000       .debug$S                   0000000180000000     ucrt:api-ms-win-crt-string-l1-1-0.dll
 0000:fffd5000       .debug$S                   0000000180000000     ucrt:api-ms-win-crt-string-l1-1-0.dll
 0000:fffd5000       .debug$S                   0000000180000000     kernel32:KERNEL32.dll
 0000:fffd5000       .debug$S                   0000000180000000     kernel32:KERNEL32.dll
 0000:fffd5000       .debug$S                   0000000180000000     kernel32:KERNEL32.dll
 0000:fffd5000       .debug$S                   0000000180000000     kernel32:KERNEL32.dll
 0000:fffd5000       .debug$S                   0000000180000000     kernel32:KERNEL32.dll
 0000:fffd5000       .debug$S                   0000000180000000     kernel32:KERNEL32.dll
 0000:fffd5000       .debug$S                   0000000180000000     kernel32:KERNEL32.dll
 0000:fffd5000       .debug$S                   0000000180000000     kernel32:KERNEL32.dll
 0000:fffd5000       .debug$S                   0000000180000000     kernel32:KERNEL32.dll
 0000:fffd5000       .debug$S                   0000000180000000     kernel32:KERNEL32.dll
 0000:fffd5000       .debug$S                   0000000180000000     kernel32:KERNEL32.dll
 0000:fffd5000       .debug$S                   0000000180000000     kernel32:KERNEL32.dll
 0000:fffd5000       .debug$S                   0000000180000000     kernel32:KERNEL32.dll
 0000:fffd5000       .debug$S                   0000000180000000     kernel32:KERNEL32.dll
 0000:fffd5000       .debug$S                   0000000180000000     kernel32:KERNEL32.dll
 0000:fffd5000       .debug$S                   0000000180000000     kernel32:KERNEL32.dll
 0000:fffd5000       .debug$S                   0000000180000000     kernel32:KERNEL32.dll
 0000:fffd5000       .debug$S                   0000000180000000     kernel32:KERNEL32.dll
 0000:fffd5000       .debug$S                   0000000180000000     kernel32:KERNEL32.dll
 0000:fffd5000       .debug$S                   0000000180000000     kernel32:KERNEL32.dll
 0000:fffd5000       .debug$S                   0000000180000000     kernel32:KERNEL32.dll
 0000:fffd5000       .debug$S                   0000000180000000     kernel32:KERNEL32.dll
 0000:fffd5000       .debug$S                   0000000180000000     kernel32:KERNEL32.dll
 0000:fffd5000       .debug$S                   0000000180000000     kernel32:KERNEL32.dll
 0000:fffd5000       .debug$S                   0000000180000000     kernel32:KERNEL32.dll
 0000:fffd5000       .debug$S                   0000000180000000     kernel32:KERNEL32.dll
 0000:fffd5000       .debug$S                   0000000180000000     kernel32:KERNEL32.dll
 0000:fffd5000       .debug$S                   0000000180000000     kernel32:KERNEL32.dll
 0001:0000146c       addRefToVerify             000000018000246c f   libStackTrace.obj
 0001:000014d8       agentThreadWrapper         00000001800024d8 f   libStackTrace.obj
 0001:00001724       file_basename              0000000180002724 f   libStackTrace.obj
 0001:00001d90       startAgentThreadWrapper    0000000180002d90 f   libStackTrace.obj
 0001:000020d0       syncDebuggeeStatus         00000001800030d0 f   libStackTrace.obj
 0001:00002370       capture_previous_context   0000000180003370 f   MSVCRT:gs_report.obj
 0001:000023e4       ?__scrt_initialize_thread_safe_statics@@YAHXZ 00000001800033e4 f   MSVCRT:thread_safe_statics.obj
 0001:000024b4       ?__scrt_uninitialize_thread_safe_statics@@YAXXZ 00000001800034b4 f   MSVCRT:thread_safe_statics.obj
 0001:00002560       $$000000                   0000000180003560     MSVCRT:amdsecgs.obj
 0001:00002590       ?dllmain_crt_dispatch@@YAHQEAUHINSTANCE__@@KQEAX@Z 0000000180003590 f   MSVCRT:dll_dllmain.obj
 0001:000025e0       ?dllmain_crt_process_attach@@YAHQEAUHINSTANCE__@@QEAX@Z 00000001800035e0 f   MSVCRT:dll_dllmain.obj
 0001:000026f8       ?dllmain_crt_process_detach@@YAH_N@Z 00000001800036f8 f   MSVCRT:dll_dllmain.obj
 0001:0000277c       ?dllmain_dispatch@@YAHQEAUHINSTANCE__@@KQEAX@Z 000000018000377c f   MSVCRT:dll_dllmain.obj
 0001:00003190       $$000000                   0000000180004190     MSVCRT:guard_dispatch.obj
 0001:000031b0       $$000000                   00000001800041b0     MSVCRT:guard_xfg_dispatch.obj
 0001:000031c6       ?fin$0@?0??dllmain_crt_process_attach@@YAHQEAUHINSTANCE__@@QEAX@Z@4HA 00000001800041c6 f   MSVCRT:dll_dllmain.obj
 0001:000031dd       ?fin$0@?0??dllmain_crt_process_detach@@YAH_N@Z@4HA 00000001800041dd f   MSVCRT:dll_dllmain.obj
 0001:000031f6       ?fin$1@?0??dllmain_crt_process_detach@@YAH_N@Z@4HA 00000001800041f6 f   MSVCRT:dll_dllmain.obj
 0001:0000320a       ?filt$0@?0??dllmain_dispatch@@YAHQEAUHINSTANCE__@@KQEAX@Z@4HA 000000018000420a f   MSVCRT:dll_dllmain.obj
 0001:00003240       __scrt_is_nonwritable_in_current_image$filt$0 0000000180004240 f   MSVCRT:utility.obj
 0002:000001e8       ?__scrt_initialize_tss_var@@3P6AHXZEA 00000001800051e8     MSVCRT:thread_safe_statics.obj
 0002:00000310       ?opcLengths@@3QBEB         0000000180005310     libStackTrace.obj
 0002:00001d28       GS_ExceptionPointers       0000000180006d28     MSVCRT:gs_report.obj
 0002:00002418       $unwind$fprintf            0000000180007418     libStackTrace.obj
 0002:00002424       $unwind$printf             0000000180007424     libStackTrace.obj
 0002:00002430       $unwind$_snprintf          0000000180007430     libStackTrace.obj
 0002:00002440       $unwind$?NewObject@JNIEnv_@@QEAAPEAV_jobject@@PEAV_jclass@@PEAU_jmethodID@@ZZ 0000000180007440     libStackTrace.obj
 0002:00002440       $unwind$nsk_lcomplain      0000000180007440     libStackTrace.obj
 0002:00002440       $unwind$nsk_ldisplay       0000000180007440     libStackTrace.obj
 0002:00002448       $unwind$Agent_Initialize   0000000180007448     libStackTrace.obj
 0002:00002448       $unwind$nsk_lvdisplay      0000000180007448     libStackTrace.obj
 0002:00002448       $unwind$_RTC_Initialize    0000000180007448     MSVCRT:initsect.obj
 0002:00002448       $unwind$_RTC_Terminate     0000000180007448     MSVCRT:initsect.obj
 0002:00002448       $unwind$?__scrt_initialize_thread_safe_statics@@YAHXZ 0000000180007448     MSVCRT:thread_safe_statics.obj
 0002:00002454       $unwind$nsk_lvcomplain     0000000180007454     libStackTrace.obj
 0002:0000246c       $unwind$nsk_ltrace         000000018000746c     libStackTrace.obj
 0002:0000246c       $unwind$__report_gsfailure 000000018000746c     MSVCRT:gs_report.obj
 0002:00002474       $unwind$Java_nsk_jvmti_unit_StackTrace_JvmtiTest_GetFrameCount 0000000180007474     libStackTrace.obj
 0002:00002474       $unwind$Java_nsk_jvmti_unit_StackTrace_JvmtiTest_RawMonitorEnter 0000000180007474     libStackTrace.obj
 0002:00002474       $unwind$Java_nsk_jvmti_unit_StackTrace_JvmtiTest_RawMonitorExit 0000000180007474     libStackTrace.obj
 0002:00002474       $unwind$Java_nsk_jvmti_unit_StackTrace_JvmtiTest_RawMonitorNotify 0000000180007474     libStackTrace.obj
 0002:00002474       $unwind$Java_nsk_jvmti_unit_StackTrace_JvmtiTest_RawMonitorWait 0000000180007474     libStackTrace.obj
 0002:00002474       $unwind$nsk_lvtrace        0000000180007474     libStackTrace.obj
 0002:00002474       $unwind$__raise_securityfailure 0000000180007474     MSVCRT:gs_report.obj
 0002:00002474       $unwind$__scrt_initialize_crt 0000000180007474     MSVCRT:utility.obj
 0002:00002474       $unwind$__scrt_initialize_onexit_tables 0000000180007474     MSVCRT:utility.obj
 0002:00002474       $unwind$__scrt_release_startup_lock 0000000180007474     MSVCRT:utility.obj
 0002:00002474       $unwind$__scrt_uninitialize_crt 0000000180007474     MSVCRT:utility.obj
 0002:00002474       $unwind$_onexit            0000000180007474     MSVCRT:utility.obj
 0002:0000247c       $unwind$nsk_lverify        000000018000747c     libStackTrace.obj
 0002:0000248c       $unwind$nsk_vprintf        000000018000748c     libStackTrace.obj
 0002:0000249c       $unwind$nsk_printf         000000018000749c     libStackTrace.obj
 0002:000024a4       $unwind$?nsk_jni_lverify@@YAHHPEAUJNIEnv_@@HQEBDH1ZZ 00000001800074a4     libStackTrace.obj
 0002:000024b8       $unwind$?nsk_jni_check_exception@@YAHPEAUJNIEnv_@@QEBDH@Z 00000001800074b8     libStackTrace.obj
 0002:000024d4       $unwind$Java_nsk_jvmti_unit_FollowReferences_FollowRefObjects_resetTags 00000001800074d4     libStackTrace.obj
 0002:000024d4       $unwind$addRefToVerify     00000001800074d4     libStackTrace.obj
 0002:000024d4       $unwind$nsk_jvmti_resetAgentData 00000001800074d4     libStackTrace.obj
 0002:000024d4       $unwind$nsk_jvmti_setFailStatus 00000001800074d4     libStackTrace.obj
 0002:000024d4       $unwind$__scrt_initialize_default_local_stdio_options 00000001800074d4     MSVCRT:default_local_stdio_options.obj
 0002:000024d4       $unwind$?dllmain_crt_dispatch@@YAHQEAUHINSTANCE__@@KQEAX@Z 00000001800074d4     MSVCRT:dll_dllmain.obj
 0002:000024d4       $unwind$DllMain            00000001800074d4     MSVCRT:dll_dllmain_stub.obj
 0002:000024d4       $unwind$__GSHandlerCheck   00000001800074d4     MSVCRT:gshandler.obj
 0002:000024d4       $unwind$?__scrt_uninitialize_thread_safe_statics@@YAXXZ 00000001800074d4     MSVCRT:thread_safe_statics.obj
 0002:000024d4       $unwind$__scrt_acquire_startup_lock 00000001800074d4     MSVCRT:utility.obj
 0002:000024d4       $unwind$__scrt_dllmain_after_initialize_c 00000001800074d4     MSVCRT:utility.obj
 0002:000024d4       $unwind$__scrt_dllmain_before_initialize_c 00000001800074d4     MSVCRT:utility.obj
 0002:000024d4       $unwind$__scrt_dllmain_crt_thread_attach 00000001800074d4     MSVCRT:utility.obj
 0002:000024d4       $unwind$__scrt_dllmain_crt_thread_detach 00000001800074d4     MSVCRT:utility.obj
 0002:000024d4       $unwind$__scrt_dllmain_uninitialize_c 00000001800074d4     MSVCRT:utility.obj
 0002:000024d4       $unwind$__scrt_dllmain_uninitialize_critical 00000001800074d4     MSVCRT:utility.obj
 0002:000024d4       $unwind$atexit             00000001800074d4     MSVCRT:utility.obj
 0002:000024dc       $unwind$nsk_jvmti_lverify  00000001800074dc     libStackTrace.obj
 0002:000024f0       $unwind$exitOnError        00000001800074f0     libStackTrace.obj
 0002:00002500       $unwind$Java_nsk_share_jvmti_ArgumentHandler_getAgentOptionsString 0000000180007500     libStackTrace.obj
 0002:00002514       $unwind$Java_nsk_jvmti_unit_FollowReferences_FollowRefObjects_getTag 0000000180007514     libStackTrace.obj
 0002:00002514       $unwind$Java_nsk_share_jvmti_DebugeeClass_checkStatus 0000000180007514     libStackTrace.obj
 0002:00002514       $unwind$agentThreadWrapper 0000000180007514     libStackTrace.obj
 0002:00002524       $unwind$startAgentThreadWrapper 0000000180007524     libStackTrace.obj
 0002:00002540       $unwind$syncDebuggeeStatus 0000000180007540     libStackTrace.obj
 0002:00002540       $unwind$__scrt_dllmain_exception_filter 0000000180007540     MSVCRT:utility.obj
 0002:00002554       $unwind$Java_nsk_share_jvmti_DebugeeClass_resetAgentData 0000000180007554     libStackTrace.obj
 0002:0000255c       $unwind$MA_checkStatus     000000018000755c     libStackTrace.obj
 0002:00002570       $unwind$Java_nsk_jvmti_unit_FollowReferences_FollowRefObjects_setTag 0000000180007570     libStackTrace.obj
 0002:00002588       $unwind$Java_nsk_jvmti_unit_FollowReferences_FollowRefObjects_addRefToVerify 0000000180007588     libStackTrace.obj
 0002:000025a4       $unwind$debug_printf       00000001800075a4     libStackTrace.obj
 0002:000025b0       $unwind$Java_nsk_jvmti_unit_StackTrace_JvmtiTest_CreateRawMonitor 00000001800075b0     libStackTrace.obj
 0002:000025c4       $unwind$Java_nsk_jvmti_unit_StackTrace_JvmtiTest_GetStackTrace 00000001800075c4     libStackTrace.obj
 0002:000025dc       $unwind$capture_previous_context 00000001800075dc     MSVCRT:gs_report.obj
 0002:000025e8       $unwind$__GSHandlerCheckCommon 00000001800075e8     MSVCRT:gshandler.obj
 0002:000025f0       $xdatasym                  00000001800075f0     MSVCRT:amdsecgs.obj
 0002:000025f4       $unwind$?dllmain_crt_process_attach@@YAHQEAUHINSTANCE__@@QEAX@Z 00000001800075f4     MSVCRT:dll_dllmain.obj
 0002:00002630       $unwind$?fin$0@?0??dllmain_crt_process_attach@@YAHQEAUHINSTANCE__@@QEAX@Z@4HA 0000000180007630     MSVCRT:dll_dllmain.obj
 0002:00002630       $unwind$?fin$0@?0??dllmain_crt_process_detach@@YAH_N@Z@4HA 0000000180007630     MSVCRT:dll_dllmain.obj
 0002:00002630       $unwind$?fin$1@?0??dllmain_crt_process_detach@@YAH_N@Z@4HA 0000000180007630     MSVCRT:dll_dllmain.obj
 0002:00002638       $unwind$?dllmain_crt_process_detach@@YAH_N@Z 0000000180007638     MSVCRT:dll_dllmain.obj
 0002:0000268c       $unwind$?dllmain_dispatch@@YAHQEAUHINSTANCE__@@KQEAX@Z 000000018000768c     MSVCRT:dll_dllmain.obj
 0002:000026b4       $unwind$?filt$0@?0??dllmain_dispatch@@YAHQEAUHINSTANCE__@@KQEAX@Z@4HA 00000001800076b4     MSVCRT:dll_dllmain.obj
 0002:000026bc       $unwind$_DllMainCRTStartup 00000001800076bc     MSVCRT:dll_dllmain.obj
 0002:000026cc       $unwind$__scrt_is_nonwritable_in_current_image 00000001800076cc     MSVCRT:utility.obj
 0002:000026ec       $unwind$__scrt_is_nonwritable_in_current_image$filt$0 00000001800076ec     MSVCRT:utility.obj
 0002:000026f4       $unwind$__scrt_fastfail    00000001800076f4     MSVCRT:utility_desktop.obj
 0002:00002704       $unwind$__security_init_cookie 0000000180007704     MSVCRT:gs_support.obj
 0002:00002710       $unwind$__isa_available_init 0000000180007710     MSVCRT:cpu_disp.obj
 0002:00002720       $xdatasym                  0000000180007720     MSVCRT:guard_dispatch.obj
 0002:00002728       $xdatasym                  0000000180007728     MSVCRT:guard_xfg_dispatch.obj
 0002:00002730       .edata                     0000000180007730     StackTrace.exp
 0002:00002758       rgpv                       0000000180007758     StackTrace.exp
 0002:000027b4       rgszName                   00000001800077b4     StackTrace.exp
 0002:00002810       rgwOrd                     0000000180007810     StackTrace.exp
 0002:0000283e       szName                     000000018000783e     StackTrace.exp
 0002:0000284d       $N00001                    000000018000784d     StackTrace.exp
 0002:0000285c       $N00002                    000000018000785c     StackTrace.exp
 0002:00002869       $N00003                    0000000180007869     StackTrace.exp
 0002:000028ae       $N00004                    00000001800078ae     StackTrace.exp
 0002:000028eb       $N00005                    00000001800078eb     StackTrace.exp
 0002:00002933       $N00006                    0000000180007933     StackTrace.exp
 0002:00002973       $N00007                    0000000180007973     StackTrace.exp
 0002:000029b0       $N00008                    00000001800079b0     StackTrace.exp
 0002:000029ea       $N00009                    00000001800079ea     StackTrace.exp
 0002:00002a21       $N00010                    0000000180007a21     StackTrace.exp
 0002:00002a54       $N00011                    0000000180007a54     StackTrace.exp
 0002:00002a8b       $N00012                    0000000180007a8b     StackTrace.exp
 0002:00002ac4       $N00013                    0000000180007ac4     StackTrace.exp
 0002:00002afc       $N00014                    0000000180007afc     StackTrace.exp
 0002:00002b36       $N00015                    0000000180007b36     StackTrace.exp
 0002:00002b6e       $N00016                    0000000180007b6e     StackTrace.exp
 0002:00002ba6       $N00017                    0000000180007ba6     StackTrace.exp
 0002:00002be1       $N00018                    0000000180007be1     StackTrace.exp
 0002:00002c0f       $N00019                    0000000180007c0f     StackTrace.exp
 0002:00002c40       $N00020                    0000000180007c40     StackTrace.exp
 0002:00002c6f       $N00021                    0000000180007c6f     StackTrace.exp
 0002:00002c9e       $N00022                    0000000180007c9e     StackTrace.exp
 0002:00002cd3       $N00023                    0000000180007cd3     StackTrace.exp
 0002:000030e2       .idata$6                   00000001800080e2     kernel32:KERNEL32.dll
 0002:00003150       .idata$6                   0000000180008150     vcruntime:VCRUNTIME140.dll
 0002:000032b2       .idata$6                   00000001800082b2     ucrt:api-ms-win-crt-runtime-l1-1-0.dll
 0002:000032d4       .idata$6                   00000001800082d4     ucrt:api-ms-win-crt-stdio-l1-1-0.dll
 0002:000032f4       .idata$6                   00000001800082f4     ucrt:api-ms-win-crt-string-l1-1-0.dll
 0003:00000000       ?codeAttributeName@@3PEBDEB 0000000180009000     libStackTrace.obj
 0003:00000008       ?lineNumberAttributeName@@3PEBDEB 0000000180009008     libStackTrace.obj
 0003:00000010       ?localVarAttributeName@@3PEBDEB 0000000180009010     libStackTrace.obj
 0003:00000018       ?localVarTypeAttributeName@@3PEBDEB 0000000180009018     libStackTrace.obj
 0003:00000020       ?stackMapAttributeName@@3PEBDEB 0000000180009020     libStackTrace.obj
 0003:00000028       ?callBytes@@3PAEA          0000000180009028     libStackTrace.obj
 0003:0000002c       ?allocBytes@@3PAEA         000000018000902c     libStackTrace.obj
 0003:0001ea08       nsk_context                0000000180027a08     libStackTrace.obj
 0003:0001ea14       redefineAttempted          0000000180027a14     libStackTrace.obj
 0003:0001ea18       redefineSucceed            0000000180027a18     libStackTrace.obj
 0003:0001ea1c       agentFailed                0000000180027a1c     libStackTrace.obj
 0003:0001ea20       context                    0000000180027a20     libStackTrace.obj
 0003:0001ead8       agentThread                0000000180027ad8     libStackTrace.obj
 0003:0001eae0       agentThreadProc            0000000180027ae0     libStackTrace.obj
 0003:0001eae8       agentThreadArg             0000000180027ae8     libStackTrace.obj
 0003:0001eaf0       agent_data                 0000000180027af0     libStackTrace.obj
 0003:0001eb00       jvmti_env                  0000000180027b00     libStackTrace.obj
 0003:0001eb08       jvm                        0000000180027b08     libStackTrace.obj
 0003:0001eb10       jni_env                    0000000180027b10     libStackTrace.obj
 0003:0001eb18       currentAgentStatus         0000000180027b18     libStackTrace.obj
 0003:0001eb1c       ?codeAttributeIndex@@3GA   0000000180027b1c     libStackTrace.obj
 0003:0001eb20       checkStatus_func           0000000180027b20     libStackTrace.obj
 0003:0001eb28       ?lineNumberAttributeIndex@@3GA 0000000180027b28     libStackTrace.obj
 0003:0001eb2c       ?localVarAttributeIndex@@3GA 0000000180027b2c     libStackTrace.obj
 0003:0001eb30       ?localVarTypeAttributeIndex@@3GA 0000000180027b30     libStackTrace.obj
 0003:0001eb34       ?stackMapAttributeIndex@@3GA 0000000180027b34     libStackTrace.obj
 0003:0001eb38       ?stackFrameOffset@@3GA     0000000180027b38     libStackTrace.obj
 0003:0001eb3c       ?mode@@3HA                 0000000180027b3c     libStackTrace.obj
 0003:0001eb40       ?orig@@3PEBEEB             0000000180027b40     libStackTrace.obj
 0003:0001eb48       ?gen@@3PEAEEA              0000000180027b48     libStackTrace.obj
 0003:0001eb50       ?inputPos@@3PEAEEA         0000000180027b50     libStackTrace.obj
 0003:0001eb58       ?endPos@@3PEBEEB           0000000180027b58     libStackTrace.obj
 0003:0001eb60       ?genPos@@3PEAEEA           0000000180027b60     libStackTrace.obj
 0003:0001eb68       ?markPos@@3PEAEEA          0000000180027b68     libStackTrace.obj
 0003:0001eb70       ?constantPool@@3PEAPEADEA  0000000180027b70     libStackTrace.obj
 0003:0001eb78       ?constantPoolSize@@3GA     0000000180027b78     libStackTrace.obj
 0003:0001eb7c       ?constantPoolCount@@3GA    0000000180027b7c     libStackTrace.obj
 0003:0001eb80       ?zeroBytes@@3PAEA          0000000180027b80     libStackTrace.obj
 0003:0001eb84       ?codeLength@@3IA           0000000180027b84     libStackTrace.obj
 0003:0001eb88       ?map@@3PEAIEA              0000000180027b88     libStackTrace.obj
 0003:0001eb90       ?widening@@3PEACEA         0000000180027b90     libStackTrace.obj
 0003:0001eb98       jvmti_caps                 0000000180027b98     libStackTrace.obj
 0003:0001ebb0       GS_ExceptionRecord         0000000180027bb0     MSVCRT:gs_report.obj
 0003:0001ec50       GS_ContextRecord           0000000180027c50     MSVCRT:gs_report.obj
 0003:0001f120       ?g_tss_cv@@3U_RTL_CONDITION_VARIABLE@@A 0000000180028120     MSVCRT:thread_safe_statics.obj
 0003:0001f128       ?g_tss_event@@3PEAXEA      0000000180028128     MSVCRT:thread_safe_statics.obj
 0003:0001f130       ?g_tss_mutex@@3U_RTL_CRITICAL_SECTION@@A 0000000180028130     MSVCRT:thread_safe_statics.obj
 0003:0001f158       ?g_sleep_condition_variable_cs@@3P6AHPEAU_RTL_CONDITION_VARIABLE@@PEAU_RTL_CRITICAL_SECTION@@K@ZEA 0000000180028158     MSVCRT:thread_safe_statics.obj
 0003:0001f160       ?g_wake_all_condition_variable@@3P6AXPEAU_RTL_CONDITION_VARIABLE@@@ZEA 0000000180028160     MSVCRT:thread_safe_statics.obj
 0003:0001f16c       ?__proc_attached@@3HA      000000018002816c     MSVCRT:dll_dllmain.obj
 0003:0001f180       ?is_initialized_as_dll@@3_NA 0000000180028180     MSVCRT:utility.obj
 0003:0001f181       ?module_local_atexit_table_initialized@@3_NA 0000000180028181     MSVCRT:utility.obj
 0003:0001f188       ?module_local_atexit_table@@3U_onexit_table_t@@A 0000000180028188     MSVCRT:utility.obj
 0003:0001f1a0       ?module_local_at_quick_exit_table@@3U_onexit_table_t@@A 00000001800281a0     MSVCRT:utility.obj
